:1000000002175902006EAE07021E15021C1653BCE1
:02001000DF32DD
:06001300020086021967DD
:06001B000200260214C8D9
:060023000219CEB2EE321C
:0E002B0002000E121D14121BD5D2AF020016D9
:0F003B00020BA5AD07AC06ECFF021B92B2ED3233
:06004B00021A71B2EC3252
:06005300021DCBB2EB32EE
:03005B00021DDEA5
:0300630002004751
:10006B00021350C0E0C083C082900C607401F0D0CA
:06007B0082D083D0E032C8
:10008300021DF1C0E0C083C082900C607402F0D006
:0600930082D083D0E032B0
:03009B0002004E12
:0300A30002005602
:0300AB00021E042E
:0B00B300021CBB12002E1200C680FBD6
:1000C30002169EE4900BC5F0900C37E0FF900BC531
:1000D300E0FEC39F5044EE75F008A42438F582E493
:1000E300340CF583E0602B900BC5E0FF75F008A49A
:1000F3002438F582E4340CF583E4F0EF75F008A4BA
:10010300243DF582E4340CF583A3E0FAA3E0F9126D
:10011300055B900BC5E004F080AE22E4FF121D3CAA
:03012300021D605A
:02012B0021DDD4
:0201330021DDCC
:02013B0021DDC4
:0201430021DDBC
:02014B0021DDB4
:0201530021DDAC
:02015B0021DDA4
:020163008078A2
:02016B008070A2
:020173008068A2
:02017B008060A2
:020183008058A2
:02018B008050A2
:020193008048A2
:02019B008040A2
:0201A3008038A2
:0201AB008030A2
:0201B3008028A2
:0201BB008020A2
:0201C3008018A2
:0201CB008010A2
:0201D3008008A2
:1001DB008000016BE709F608DFFA8046E709F208B1
:1001EB00DFFA803E88828C83E709F0A3DFFA803246
:1001FB00E309F608DFFA8078E309F208DFFA80708A
:10020B0088828C83E309F0A3DFFA806489828A8376
:10021B00E0A3F608DFFA805889828A83E0A3F2080C
:10022B00DFFA804C80D280FA80C680D4806980F25D
:10023B008033801080A680EA809A80A880DA80E2E2
:10024B0080CA803389828A83ECFAE493A3C8C5827F
:10025B00C8CCC583CCF0A3C8C582C8CCC583CCDFC2
:10026B00E9DEE7800D89828A83E493A3F608DFF940
:10027B00ECFAA9F0EDFB2289828A83ECFAE0A3C8A1
:10028B00C582C8CCC583CCF0A3C8C582C8CCC583F6
:10029B00CCDFEADEE880DB89828A83E493A3F20871
:1002AB00DFF980CC88F0EF60010E4E60C388F0ED73
:1002BB002402B4040050B9F582EB2402B4040050BC
:1002CB00AF232345822390022F73BB010689828AB9
:1002DB0083E0225002E722BBFE02E32289828A835B
:1002EB00E49322BB010CE58229F582E5833AF58381
:1002FB00E0225006E92582F8E622BBFE06E92582BC
:10030B00F8E222E58229F582E5833AF583E493222C
:10031B00BB010689828A83F0225002F722BBFE01C1
:10032B00F322BC000BBE0029EF8DF084FFADF02251
:10033B00E4CCF875F008EF2FFFEE33FEEC33FCEE58
:10034B009DEC984005FCEE9DFE0FD5F0E9E4CEFD4B
:10035B0022EDF8F5F0EE8420D21CFEADF075F0081E
:10036B00EF2FFFED33FD4007985006D5F0F222C377
:10037B0098FD0FD5F0EA22C5F0F8A3E028F0C5F000
:10038B00F8E582158270021583E038F022A3F8E0BD
:10039B00C5F025F0F0E582158270021583E0C838B0
:1003AB00F0E822BB0110E58229F582E5833AF5835B
:1003BB00E0F5F0A3E0225009E92582F886F008E683
:1003CB0022BBFE0AE92582F8E2F5F008E222E5837A
:1003DB002AF583E993F5F0A3E9932275F00875826A
:1003EB0000EF2FFFEE33FECD33CDCC33CCC58233B4
:1003FB00C5829BED9AEC99E58298400CF582EE9BB9
:10040B00FEED9AFDEC99FC0FD5F0D6E4CEFBE4CDD6
:10041B00FAE4CCF9A88222B800C1B90059BA002D70
:10042B00EC8BF084CFCECDFCE5F0CBF97818EF2F29
:10043B00FFEE33FEED33FDEC33FCEB33FB10D70358
:10044B00994004EB99FB0FD8E5E4F9FA227818EF01
:10045B002FFFEE33FEED33FDEC33FCC933C910D760
:10046B00059BE99A4007EC9BFCE99AF90FD8E0E46D
:10047B00C9FAE4CCFB2275F010EF2FFFEE33FEED43
:10048B0033FDCC33CCC833C810D7079BEC9AE89913
:10049B00400AED9BFDEC9AFCE899F80FD5F0DAE4F5
:1004AB00CDFBE4CCFAE4C8F922EB9FF5F0EA9E42CF
:1004BB00F0E99D42F0EC6480C864809845F022EB33
:1004CB009FF5F0EA9E42F0E99D42F0E89C45F02250
:1004DB00E8600FECC313FCED13FDEE13FEEF13FFFF
:1004EB00D8F122BB010DE58229F582E5833AF5832C
:1004FB0002056E5007E92582F8020561BBFE07E98C
:10050B002582F802057AE58229F582E5833AF5839F
:10051B00020587ECF0A3EDF0A3EEF0A3EFF022A819
:10052B00828583F0D083D0821205411205411205DA
:10053B0041120541E473E493A3C583C5F0C583C899
:10054B00C582C8F0A3C583C5F0C583C8C582C822C0
:10055B008A838982E473E6FB08E6F908E6FA08E683
:10056B00CBF822E0F8A3E0F9A3E0FAA3E0FB22E248
:10057B00FB08E2F908E2FA08E2CBF822E493F874FC
:10058B000193F9740293FA740393FB22F8E0FBA333
:10059B00A3E0F925F0F0E582158270021583E0FAED
:1005AB0038F022EBF0A3EAF0A3E9F022D083D0825B
:1005BB00F8E4937012740193700DA3A393F8740174
:1005CB0093F5828883E4737402936860EFA3A3A30B
:1005DB0080DFE50824D2F582E4340BF583E00508CF
:1005EB0022900BCF300703900BD2E475F00112056C
:1005FB00970202D52000E97F2ED2008018EF540F0E
:10060B002490D43440D4FF30040BEF24BFB41A0031
:10061B0050032461FFE50960021509050CE50C7018
:10062B0002050B30070E900BCFE475F00112059706
:10063B00EF02031B0200067403D2078003E4C20718
:10064B00F508900BCF1205AEE4F509F50BF50CE5AB
:10065B000960077F2012062080F5750AFFC201C2D0
:10066B0000C202C203C205C206C2081205ECFF702B
:10067B000D3007057F00120631AF0CAE0B22B425EF
:10068B005FC2D5C2041205ECFF24D0B40A00501A85
:10069B0075F00A780930D50508B6FF0106C6A42601
:1006AB00F620D5047002D20380D924CFB41A00EF00
:1006BB005004C2E5D204020832D20180C6D20080B7
:1006CB00C0D20280BCD2D580BAD20580B47F2012B2
:1006DB0006202002077401B5090040F11205DDFF69
:1006EB0012062002065AD208D20680951205DDFBAF
:1006FB001205DDFA1205DDF94A4B700679037A090A
:10070B007BFF20022EE509602A7E008E8275830016
:10071B001202EE60060EEE650A70F0C2D5EBC0E079
:10072B00EAC0E0E9C0E0EE120879D0E0F9D0E0FAD7
:10073B00D0E0FB1202D5FF60AAEBC0E0EAC0E0E913
:10074B00C0E0120620D0E02401F9D0E03400FAD04A
:10075B00E0FBE50A0460DCD50AD980877BFF7A08C9
:10076B007975D202809C791080027908C206C20882
:10077B008008D2D5790A8004790AC2D5E50A0470BB
:10078B0002F50AE4FAFDFEFF1205DDFC7B082001F1
:10079B00131205DDFD7B1030000A1205DDFE12057C
:1007AB00DDFF7B20EC3382D592D55013C3E43000B0
:1007BB00069FFFE49EFEE42001039DFDE49CFCE408
:1007CB00CBF8C201EC700CCFCECDCCE824F8F8708E
:1007DB00F38017C3EF33FFEE33FEED33FDEC33FC49
:1007EB00EB33FB994002FB0FD8E9EB300105F8D056
:1007FB00E0C448B201C0E00AEC4D4E4F78207B00BC
:10080B0070C2EAB50A0040BCC0E012087BD0F0D041
:10081B00E0200104C4C0E0C4B201C0F0120609D04C
:10082B00F0D5F0EB02065A1205B706F753077158CD
:10083B0006C84C06C44207754F077D44077D490621
:10084B00DD43078355076746076745076747092356
:10085B005006CC2D06D02E06F32B06D42306F12002
:10086B00090C2A068C48000006EB3F3F3F00790A33
:10087B00A2D5200314300509B910020404B90801EC
:10088B0004A2D52006025001042002689202B50989
:10089B00005034C0E07F203003197F30A202720673
:1008AB007205500F1208D2C202C206C205C2087FDF
:1008BB0030800F300503E9C0E0120620300503D06D
:1008CB00E0F9D0E0B509CC3005177F30B9100C1228
:1008DB0006207F583004077F788003B9080312067F
:1008EB00203002057F2D0206207F202008F87F2B69
:1008FB002006F322920280CF286E756C6C2900D2F1
:10090B00011205DD3001F8C201780930D50108F676
:10091B0002068C2D504349581205DD2403B4050003
:10092B004001E490091E93120611743A120611D27B
:10093B0003750904020771AD07ED707EC28C1202BC
:10094B00D5FEC394037480948040037FFF22E58916
:10095B0054FC4EF5899000011202EEFED394027402
:10096B0080948040037FFF22EEFF7E007006538E43
:10097B007F5389FBEF64014E7006438E805389FBD6
:10098B00EF64024E70034389049000021202EEFFE3
:10099B00E58F54FE4FF58F9000031203AEE5F0F593
:1009AB008C9000031203AEF58A9000051202EE70D4
:1009BB0004C28C8002D28C7F0022ED6401600302A2
:1009CB000A52C28E1202D5FEC394037480948040E7
:1009DB00037FFF22EEC454F0FFE58954CF4FF58916
:1009EB009000011202EEFED39402748094804003B7
:1009FB007FFF22EEFF7E007006538EBF5389BFEF41
:100A0B0064014E7006438E405389BFEF64024E70F3
:100A1B00034389409000021202EE25E0FFE58F545C
:100A2B00FD4FF58F9000031203AEE5F0F58D9000AE
:100A3B00031203AEF58B9000051202EE7004C28E0A
:100A4B008002D28E7F0022ED64027061538EEF9094
:100A5B0000011202EEFF7E007006538EFB538EF7E1
:100A6B00EF64014E7006438E04538EF7EF64024E13
:100A7B007003438E089000021202EE25E025E0FF82
:100A8B00E58F54FB4FF58F9000031203AEE5F0F5A5
:100A9B00D69000031203AEF5D79000051202EEC4F8
:100AAB0054F0FFE58E54EF4FF58E7F0022ED64037B
:100ABB00706953D1F79000011202EEFED3940274C9
:100ACB0080948040037FFF22EEFF7E00700653D19F
:100ADB00FD53D1FBEF64014E700643D10253D1FBA2
:100AEB00EF64024E700343D1049000021202EEFF3A
:100AFB00E5D154FE4FF5D19000031203AEE5F0F5AE
:100B0B00D49000031203AEF5D59000051202EE331C
:100B1B00333354F8FFE5D154F78076ED64047077E6
:100B2B0053D17F9000011202EEFD7C00D39402742E
:100B3B0080948040037FFF22ED4C700653D1DF532E
:100B4B00D1BF9000011202EE6401700643D1205315
:100B5B00D1BF9000011202EE6402700343D14090AA
:100B6B0000021202EEC454F0FFE5D154EF4FF5D161
:100B7B009000031203AEFDACF0ECF5D2AF058FD3B2
:100B8B009000051202EEC43333335480FFE5D15489
:100B9B007F4FF5D17F00227FFF22C0E0C083C08250
:100BAB00C0D075D000C002C004C005C006C007305D
:100BBB00D87BC2D8AFDAC3EF944874809480401FBF
:100BCB00900C19E0FEA3E0FF900C22E02FF0900CAC
:100BDB0021E03EF0E0FEA3E0F5EAEEF5FA804EE50B
:100BEB00DA54116048900C2FE0FFA3E0900C27CF54
:100BFB00F0A3EFF0AFFA900C2FE4F0A3EFF0E0FED0
:100C0B00ADEA7C00E42DFFEC3E900C2FF0A3EFF04F
:100C1B00900C27E0FEA3E0FFC3900C30E09FFF9009
:100C2B000C2FE09E900C21F0A3EFF0D21B30D97B60
:100C3B00C2D9AFDBC3EF944874809480401F900CF3
:100C4B001BE0FEA3E0FF900C24E02FF0900C23E0C0
:100C5B003EF0E0FEA3E0F5EBEEF5FB804EE5DB545A
:100C6B00116048900C31E0FFA3E0900C29CFF0A36A
:100C7B00EFF0AFFB900C31E4F0A3EFF0E0FEADEB47
:100C8B007C00E42DFFEC3E900C31F0A3EFF0900CC8
:100C9B0029E0FEA3E0FFC3900C32E09FFF900C31E4
:100CAB00E09E900C23F0A3EFF0D21C30DA7BC2DA7B
:100CBB00AFDCC3EF944874809480401F900C1DE010
:100CCB00FEA3E0FF900C26E02FF0900C25E03EF009
:100CDB00E0FEA3E0F5ECEEF5FC804EE5DC54116094
:100CEB0048900C33E0FFA3E0900C2BCFF0A3EFF078
:100CFB00AFFC900C33E4F0A3EFF0E0FEADEC7C0026
:100D0B00E42DFFEC3E900C33F0A3EFF0900C2BE0B6
:100D1B00FEA3E0FFC3900C34E09FFF900C33E09EEA
:100D2B00900C25F0A3EFF0D21D20DB03020DC8AD14
:100D3B00BA43BA80C2DB90FD54E0C39448748094EC
:100D4B00804021900C1FE0FEA3E0FF900C14E02FDD
:100D5B00F0900C13E03EF0E0FEA3E090FD55F0EEBA
:100D6B00A3F0805590FD54E05411604D900C35E08C
:100D7B00FFA3E0900C2DCFF0A3EFF090FD56E0FF1A
:100D8B00900C35E4F0A3EFF0E0FE90FD55E07A0017
:100D9B002400FFEA3E900C35F0A3EFF0900C2DE011
:100DAB00FEA3E0FFC3900C36E09FFF900C35E09E56
:100DBB00900C13F0A3EFF0D21EAF058FBA30DF0209
:100DCB00C2DFD007D006D005D004D002D0D0D0825D
:100DDB00D083D0E032F0900BDBE0900BE9F0900B7E
:100DEB00D3E0FAA3E0FB900BDFEEF0A3EFF0900B58
:100DFB00E3EAF0A3EBF0900BE1ECF0A3EDF090063F
:100E0B0014E0FFA3E0900BEDCFF0A3EFF0900BE716
:100E1B00E024E0F0A3E0F9C313FF7E00900BDFE0CA
:100E2B00FAA3E02FFFEE3ACF24FFFBEF34FFFAE9F2
:100E3B00FFA3E0F8A3E02FFFEE38CF24FFCF34FF62
:100E4B00900BF5F0A3EFF0900BDFE0FEA3E0FF12A9
:100E5B0018F0900BE9E06003020F01900BEBF090A0
:100E6B000BE8E0FF900BEBE0FEC39F4003020FC1CA
:100E7B00EF640C7017900BE7E075F00CA4242CF5C5
:100E8B0082E5F0341EF583E5822E801A900BEBE0A1
:100E9B00FF900BE7E075F010A424A0F582E5F03489
:100EAB0022F583E5822FF582E43583F583E4939075
:100EBB000BEAF0E4900BECF0900BE8E0C313FF901F
:100ECB000BECE0C39F5026900BEAE030E005900B53
:100EDB00E38003900BE5E0FEA3E0FF12003E900BD6
:100EEB00EAE0C313F0900BECE004F080CB900BEB3B
:100EFB00E004F0020E6AE4900BEBF0900BE8E0FFDD
:100F0B00900BEBE0FEC39F4003020FC1EF640C702C
:100F1B0017900BE7E075F00CA4242CF582E5F03468
:100F2B001EF583E5822E801A900BEBE0FF900BE70A
:100F3B00E075F010A424A0F582E5F03422F583E5EA
:100F4B00822FF582E43583F583E493900BEAF0E48A
:100F5B00900BECF0900BE8E0C313FF900BECE0FE72
:100F6B00C39F5049900BE3E0FDA3E0900614CDF036
:100F7B00A3EDF0900BEAE030E024EEFF900BE0E005
:100F8B002FFF900BDFE03400FE900BEBE0FD900B9E
:100F9B00E2E02DFD900BE1E03400FC121CEA900B1B
:100FAB00EAE0C313F0900BECE004F080A7900BEB9E
:100FBB00E004F0020F06900BEDE0FFA3E0900614A7
:100FCB00CFF0A3EFF0900601E024FFFB900600E0CA
:100FDB0034FFFA900617E024FFFE900616E034FF6C
:100FEB00900BF5F0A3CEF0E4FDFCFFFE0218F0121F
:100FFB001D7F7F967E00121DB47DF07C787FE512FD
:10100B001DA27D007C017F01121DA27D007C077F4C
:10101B0002121DA27D307C107F03121DA2E4FDFC89
:10102B007F04121DA27402FDFC7F08121DA2E4FDB9
:10103B00FC7F09121DA2E4FD7F0A121DA2E4FD7FB5
:10104B000C121DA2E4FD7F0D121DA2E4FD7F0F12F9
:10105B001DA2E4FD7F10121DA27D077F11121DA2A0
:10106B00E4FD7F12121DA2E4FD7F13121DA2E4FD0D
:10107B007F07121DA27D907C167F10121DA27D276B
:10108B007C027F11121DA27F0A7E00121DB47D9D72
:10109B007C007F12121DA27F0A7E00121DB47D0000
:1010AB007C197F13121DA27F0A7E00121DB47D25B1
:1010BB007C007F29121DA27D0D7F2B121DA27D07A7
:1010CB007F30121DA27403FDFC7F31121DA27D0324
:1010DB007C007F32121DA27D067C027F35121DA281
:1010EB007D087C007F36121DA27D067C047F3712A3
:1010FB001DA27D041C7F38121DA27D077C007F3949
:10110B00121DA27D027C067F3C121DA27D087C0075
:10111B007F3D121DA2E4FD7F50121DA27DEF7F517A
:10112B00121DA2E4FD7F52121DA27D3F0C7F5312B4
:10113B001DA27D007CA77F60121DA27D017C007F1C
:10114B0061121DA2E4FD7F6A121DA2E4FD7F8012D5
:10115B001DA2E4FD7F81121DA2E4FD7F82121DA260
:10116B00E4FD7F83121DA2E4FD7F84121DA2E4FD2A
:10117B007F85121DA27D107F90121DA27D007C0623
:10118B007F92121DA27D337C017F07121DA27D224F
:10119B001CE4FF121DA29006007401F0A37440F032
:1011AB00900616E4F0A374F0F07D387C107F0312E8
:1011BB001DA2E4FDFC7F01021DA2900BD1ECF0A35C
:1011CB00EDF0A3EAF0A3EBF0900BCFEEF0A3EFF072
:1011DB00900BDCEEF0A3EFF0E4A3F0900BD7E0FB69
:1011EB00A3E0FAA3E0F91202D5700302134F900BA0
:1011FB00DEE06003021330900BDAE0FFC313FDC394
:10120B00900601E09DFD900600E09400FCD3900B4E
:10121B00D0E09D900BCFE09C400302134FC3900690
:10122B0017E09FFF900616E09400FED3900BD2E0E0
:10123B009F900BD1E09E400302134F1202D5FF7E0D
:10124B0000D39480748094804008900BDE7401F07E
:10125B008089EF640D4E702E900BDAE0FF900BD26D
:10126B00E02FF0900BD1E03400F0900BDCE0FFA30B
:10127B00E0900BCFCFF0A3EFF0900BD8E475F0011B
:10128B00120382021323900BDAE0D3941074809430
:10129B0080900BCFE0FE4038A3E0FFA3E0FCA3E07F
:1012AB00FD900BD5E0FBA3E0900BE5CBF0A3EBF0AF
:1012BB00900BD7E0FBA3E0FAA3E0F91202D5900B59
:1012CB00E7F0A37410120DE0900BD0E024088040DF
:1012DB00A3E0FFA3E0FCA3E0FD900BD5E0FBA3E0B4
:1012EB00900BE5CBF0A3EBF0900BD7E0FBA3E0FA70
:1012FB00A3E0F91202D5900BE7F0900BDAE0900B1C
:10130B00E8120DE0900BDAE0C313FF900BD0E02F47
:10131B00F0900BCFE03400F0900BD8E475F0011295
:10132B0003820211E6900BD8E475F002120382904F
:10133B000BDAE0FF900BD0E02FF0900BCFE03400F6
:10134B00F00211E622C0E0C083C082C0D075D0008D
:10135B00C007AFBA43BA8090FA12E030E006E0540F
:10136B00FEF0D22390FA02E030E014E054FEF0D20B
:10137B0024301204C212D214301104C211D21390B1
:10138B00FA32E030E006E054FEF0D20C90FA32E094
:10139B0030E204E054FBF090FA3AE030E006E0541F
:1013AB00FEF0D20990FA3AE030E104E054FDF090FF
:1013BB00FA42E030E006E054FEF0D20E90FA42E042
:1013CB0030E204E054FBF090FA4AE030E006E054DF
:1013DB00FEF0D20A90FA4AE030E104E054FDF090BE
:1013EB00FA52E030E006E054FEF0D20F90FA52E0F1
:1013FB0030E204E054FBF090FA5AE030E006E0549F
:10140B00FEF0D20B90FA5AE030E104E054FDF0907C
:10141B00FA62E030E006E054FEF0D21090FA62E09F
:10142B0030E204E054FBF090FA6AE030E006E0545E
:10143B00FEF0D20D90FA6AE030E104E054FDF0903A
:10144B00FA22E030E011E054FEF0E5CE30E406D2B3
:10145B0016D2A28002D21590FA22E030E104E054B9
:10146B00FDF090FA22E030E204E054FBF090FE53E2
:10147B00E030E004E4F0C21F90FA72E030E031306B
:10148B002009C22090FA71E4F08020900613E0242A
:10149B00FFF0900612E034FFF0E07002A3E090FA48
:1014AB00717005F0D2B4800374A0F090FA72E4F07E
:1014BB008FBAD007D0D0D082D083D0E03278C57C21
:1014CB000B7D017BFF7A2879907E007F0A1202AF99
:1014DB00900600E0FAA3E0FB900616E0FFA3E09075
:1014EB000BD5CFF0A3EFF074FFA3F01215DD30B4E2
:1014FB00FD43BA8090FA737401F053BA7F12011E48
:10150B00900BD274FFF0A3741EF0A37424F0A3EE1F
:10151B00F0A3EFF07B017A0B79C5120642900BD545
:10152B0074FFF0A374E0F0A37401F0A3740BF0A3A9
:10153B0074C5F0A37410F0A37401F07B1F7A007DC7
:10154B00197C007F327E001211C543BA8090FA736A
:10155B0074FFF053BA7F7F207E03121DB4900600F8
:10156B00E0FAA3E0FB900616E0FFA3E0900BD5CFCB
:10157B00F0A3EFF0A374F8F0A3E4F01215E07F20D2
:10158B007E03121DB4900600E0FAA3E0FB90061652
:10159B00E0FFA3E0900BD5CFF0A3EFF0A37407F01F
:1015AB0074E01215DD7F207E03121DB4900600E05F
:1015BB00FAA3E0FB900616E0FFA3E0900BD5CFF06B
:1015CB00A3EFF0A3E4F0741F1215DD7F207E03025E
:1015DB001DB4A3F0E4FDFCFFFE900BCFEEF0A3EFE8
:1015EB00F0A3ECF0A3EDF0900BCFE0FEA3E0FFC374
:1015FB00EB9FFFEA9ECF2401CF3400900BDBF0A3CF
:10160B00EFF0900BD1E0FEA3E0FFC3900BD6E09F71
:10161B00FF900BD5E09ECF2401CF3400900BDDF073
:10162B00A3EFF0900BD1E0FCA3E0FD900BD5E0FF16
:10163B00A3E0900BF5CFF0A3EFF0900BCFE0FEA360
:10164B00E0FF1218F0E4900BD9F0A3F0FDFC900B27
:10165B00D7E0FAA3E0FBED25E0FFEC33FE74002F9F
:10166B00F58274043EF583EAF0A3EBF00DBD0001A7
:10167B000CE4B505D9ECB401D59006127402F0A3B5
:10168B007458F0C2B443BA8090FA71E044A0F0539E
:10169B00BA7F22C0E0C083C082C0D075D000C00525
:1016AB00C006C007AFBA43BA8090FE84E030E607AD
:1016BB00E054BFF002174890FE84E030E53BE05465
:1016CB00DFF0900C59E06004E4F08071900C58E06E
:1016DB00600DE4F090FE87E0900C5AF0E0803790BC
:1016EB00FE87E0FE900C5AE0FD04F074482DF58265
:1016FB00E4340CF583EEF0804490FE84E030E42675
:10170B00E054EFF0E030E10890FE8674FFF0802D9E
:10171B00900C5AE004F02448F582E4340CF583E095
:10172B0090FE86F0801790FE84E030E310E054F7D3
:10173B00F0900C597401F0900C58F0D2268FBAD05F
:10174B0007D006D005D0D0D082D083D0E032787FBE
:10175B00E4F6D8FD7581240217A00200B6E493A32A
:10176B00F8E493A34003F68001F208DFF48029E448
:10177B0093A3F85407240CC8C333C4540F4420C894
:10178B00834004F456800146F6DFE4800B0102042B
:10179B000810204080901C87E47E019360BCA3FF5F
:1017AB00543F30E509541FFEE493A360010ECF5460
:1017BB00C025E060A840B8E493A3FAE493A3F8E44F
:1017CB0093A3C8C582C8CAC583CAF0A3C8C582C8BB
:1017DB00CAC583CADFE9DEE780BEE4FF900C37E0C1
:1017EB00FEEFC39E507AEF75F008A42439F582E41E
:1017FB00340CF583E0FCA3E04C6061EF75F008A4BA
:10180B002439F582E4340CF58374FFF5F01203826E
:10181B00EF75F008A42439F582E4340CF583E0FC71
:10182B00A3E04C7037EF75F008A4243BF582E43449
:10183B000CF583E0FCA3E0FDEF75F008A42439F56B
:10184B0082E4340CF583ECF0A3EDF0EF75F008A413
:10185B002438F582E4340CF5837401F00F0217E79A
:10186B002243BA8090FE53E4F09000011202EE6422
:10187B000190FE507006E04401F08004E054FEF04D
:10188B009000021202EE640290FE507006E04402D9
:10189B00F08004E054FDF09000031202EEFFD394AD
:1018AB000774809480500EEF25E025E0FF90FE51E9
:1018BB00E054E34FF09000041202EEFFD394037454
:1018CB00809480500890FE51E054FC4FF01202D5EA
:1018DB00640190FE527006E04480F08004E0547F77
:1018EB00F053BA7F22900BEFEEF0A3EFF0AE04AF04
:1018FB0005900BF7EEF0A3EFF0900BF5E0FFA3E0F4
:10190B00900BFBCFF0A3EFF0900BEFE0FFA3E09079
:10191B000BF9CFF0A3EFF0AF03900BFDEAF0A3EFC1
:10192B00F07F50121DA2900BFBE0FCA3E0FD7F515A
:10193B00121DA27F52121D9A900BFDE0FCA3E0FD3D
:10194B007F53121DA2900BF7E0FCA3E0FD7F20124A
:10195B001DA27F21121D9A7F22021D3C75950075D9
:10196B0096FF53B10F43B2F053B3FD43B402900B48
:10197B00C57401F0E4A3F0A3F0A37402F0A314F078
:10198B00FB7A0B79C512186CE4FD7F01121C519088
:10199B000BCA7401F0900BCF74FFF0900BCD740455
:1019AB00F0A37400F0900BCB7406F0A37402F07BE1
:1019BB00017A0B79CA121ABEE4FBFD7F01121B08D8
:1019CB00020FFAC0E0C083C082C0D075D000C00740
:1019DB00309831C29890081EE0702990081CE0C323
:1019EB009480748094804002E4F090081CE0FF0423
:1019FB00F0741F2FF582E43408F583E599F0900815
:101A0B001D7405F0309907C29990081BE4F0D007BC
:101A1B00D0D0D082D083D0E032EFFBD3940174804E
:101A2B0094805009EB7004C2A98002D2A9EDFF7E0D
:101A3B0000D39403748094805029EF700553B7FD45
:101A4B00C2B9EF64014E700553B7FDD2B9EF640212
:101A5B004E700543B702C2B9EF64034E700543B72E
:101A6B0002D2B97F0022C0E0C083C082C0D075D043
:101A7B0000C007E5CE30E404C2258029900C61E05C
:101A8B00C39480748094804002E4F0900C61E0FF7A
:101A9B0004F074E12FF582E4340AF583E5CFF0907E
:101AAB000AE07405F075CDC0D007D0D0D082D083BA
:101ABB00D0E03243BA8090FA72E4F0900001120346
:101ACB00AEFF90FA77E5F0F0A3EFF090000312036E
:101ADB00AEFF90FA75E5F0F0A3EFF090000512025F
:101AEB00EE90FA73F01202D5640190FA717006E071
:101AFB004480F08004E0547FF053BA7F2243BA80D5
:101B0B0090FA70E054F0F0EDD3940374809480500D
:101B1B000BE0FEED25E025E0FDEE4DF0EBD394035D
:101B2B0074809480500690FA70E04BF0EF64019053
:101B3B00FA707006E04480F08004E0547FF053BAF2
:101B4B007F7F002243BA8090FE54EFF053BA7FC2DE
:101B5B00B4D21F43BA8090FE52E054F84484F05341
:101B6B00BA7F201FFD43BA8090FE54EDF053BA7F2D
:101B7B00D21F43BA8090FE52E054F84484F053BA1B
:101B8B007F201FFDD2B42243BA8090FE54EFF05356
:101B9B00BA7FC2B4D21F43BA8090FE52E054F844CD
:101BAB0085F053BA7F201FFD43BA8090FE54EDF0B1
:101BBB0053BA7FD21F43BA8090FE52E054F844854B
:101BCB00F053BA7F201FFDD2B42253A23F53BAFE6B
:101BDB0053BAFD53BAFBE5A254F34404F5A243BA3E
:101BEB008090FE51E0549F4420F053BA7F43BA805B
:101BFB0090FE50E054F3F053BA7F53A2CF43BA8018
:101C0B0090FF14E054E7F053BA7F22C0E0C0F0C05D
:101C1B0083C082C0D075D000C000C001C002C00319
:101C2B00C004C005C006C0071217E5D007D006D008
:101C3B0005D004D003D002D001D000D0D0D082D0B8
:101C4B0083D0F0D0E03243BA8090FE50E054CFF016
:101C5B00EDD3940374809480500AE0FEEDC454F0ED
:101C6B00FDEE4DF0EF640190FE507006E04480F005
:101C7B008004E0547FF053BA7F7F0022480C380079
:101C8B0000010001FF001E410C3701410C5E0041B9
:101C9B000ADF00C123C124420614000050060200D3
:101CAB0011002200330044005500660077008800C5
:101CBB00C0E0C083C082C0D075D000C007AFBA43AC
:101CCB00BA80E5F630E30353F6F790FF05E06002C8
:101CDB00E4F08FBAD007D0D0D082D083D0E032AB33
:101CEB0007AA068D828C83C006C007AE83AF829095
:101CFB000BF5EEF0A3EFF0D007D0061218F090061C
:101D0B0014E0FEA3E0FF02003EE4900BC5F0A30439
:101D1B00F0E4A3F0A374A9F0A3749AF0A37401F0F8
:101D2B00FB7A0B79C5E4FF120942E4FD7F01021A2D
:101D3B002443BA8090FE54EFF053BA7FC2B4D21F43
:101D4B0043BA8090FE52E054F84484F053BA7F209B
:101D5B001FFDD2B422C2B4D22043BA8090FA71E0F4
:101D6B004488F053BA7F2020FDD2B4900602E0FEE7
:101D7B00A3E0FF22D2B47F327E00121DB4C2B57F26
:101D8B00967E00121DB4D2B57F327E00021DB49038
:101D9B000BF9E0FCA3E0FDAB05AA04AD07E4FF12D1
:101DAB001B4FEAFFAD03021B927DA37C08ED1D7058
:101DBB00011C144C70F7EF1F70011E144E70EA22B9
:101DCB00C0E0C083C082900C607403F0D082D083DB
:101DDB00D0E032C0E0C083C082900C607404F0D0BD
:101DEB0082D083D0E032C0E0C083C082900C60749C
:101DFB0005F0D082D083D0E032C0E0C0D053E6BF34
:101E0B00E5E61392C7D0D0D0E0328F9990081B74BF
:101E1B0001F090081BE070FA2249443A307825789B
:101E2B0000000000000000000000000000000004A3
:101E3B0004040404040004000000140A0A00000057
:101E4B000000000000000014143F140A3F0A0A00AF
:101E5B000000041E1505060C14150F0400000012DB
:101E6B00150D0A142C2A1200000000040A0A1E1574
:101E7B0015093600000002020100000000000000FE
:101E8B0000002010080808080808102000000204B1
:101E9B0008080808080804020000000004150E0ECC
:101EAB00150400000000000404041F0404040000D7
:101EBB000000000000000000000002020100000012
:101ECB0000001F00000000000000000000000000E8
:101EDB0000000200000010080808040402020201BE
:101EEB000000000E1111111111110E000000000461
:101EFB000604040404040E000000000E1111080473
:101F0B0002011F000000000E11100C1010110E002A
:101F1B00000000080C0A0A091E0818000000001F28
:101F2B0001010F1010110E000000000E09010F111E
:101F3B0011110E000000001F090804040404040022
:101F4B000000000E11110E1111110E000000000EF9
:101F5B001111111E10120E000000000000040000F1
:101F6B000000040000000000000004000000040456
:101F7B0000002010080402040810200000000000DC
:101F8B00001F00001F0000000000020408102010BA
:101F9B00080402000000000E1111080404000400E4
:101FAB000000000E111915151D011E000000000484
:101FBB00040C0A0A1E1233000000000F12120E123C
:101FCB0012120F000000001E1101010101110E0081
:101FDB000000000F1212121212120F000000001F4D
:101FEB00120A0E0A02121F000000001F120A0E0A2C
:101FFB00020207000000001C1201013911120C0033
:10200B000000003312121E12121233000000001FC8
:10201B000404040404041F000000003E0808080820
:10202B000808090700000037120A060A0A123700CF
:10203B00000000070202020202223F000000001B08
:10204B001B1B1B15151515000000003B1216161A4D
:10205B001A1217000000000E1111111111110E00B0
:10206B000000000F12120E02020207000000000E09
:10207B001111111117190E180000000F12120E0A70
:10208B00121237000000001E1101060810110F007C
:10209B000000001F1504040404040E0000000033AC
:1020AB001212121212120C000000003312120A0A42
:1020BB000C0404000000001515150E0A0A0A0A008C
:1020CB000000001B0A0A04040A0A1B000000001B84
:1020DB000A0A040404040E000000001F090804048B
:1020EB0002121F0000001C04040404040404041C5A
:1020FB0000000202020404080808100000000E0889
:10210B00080808080808080E0000040A0000000070
:10211B0000000000000000000000000000000000B4
:10212B003F00040000000000000000000000000061
:10213B0000000C121C123C000000000302020E12E5
:10214B0012120E000000000000001C1202021C0004
:10215B000000001810101C1212123C0000000000AE
:10216B0000000C121E021C000000003804041E04A8
:10217B0004041E000000000000003C120C021E2292
:10218B001C00000302020E121212370000000004A2
:10219B000000060404040E000000000800000C08F8
:1021AB00080808080700000302023A0A0E1237005B
:1021BB00000000070404040404041F0000000000D6
:1021CB0000000F15151515000000000000000F1280
:1021DB00121237000000000000000C1212120C004B
:1021EB000000000000000F1212120E020700000088
:1021FB0000001C1212121C103800000000001B06FD
:10220B00020207000000000000001E020C101E005E
:10221B000000000004040E04040418000000000079
:10222B0000001B1212123C000000000000003712CD
:10223B000A0C040000000000000015150E0A0A002D
:10224B000000000000001B0A040A1B000000000035
:10225B00000037120A0C04040300000000001E08E3
:10226B0004041E00000018080808040808080818D1
:10227B0000080808080808080808080808000604E9
:10228B0004040804040404060002251800000000DE
:10229B000000000000000000000000000000000033
:1022AB0000000000000000000808080808080800EB
:1022BB00001818000000486C2412000000000000F9
:1022CB0000000000000000002424247F1212127F63
:1022DB0012121200000000081C2A2A0A0C182828C7
:1022EB002A2A1C080800000022251515152A585407
:1022FB0054542200000000000C1212120A762529F9
:10230B0011916E000000060604030000000000009F
:10231B000000000000004020101008080808080802
:10232B0010102040000002040808101010101010AC
:10233B0008080402000000000008086B1C1C6B0856
:10234B00080000000000000000080808087F0808CB
:10235B000808000000000000000000000000000062
:10236B0000060604030000000000000000FE000051
:10237B000000000000000000000000000000000052
:10238B0000060600000000804040202010100808C6
:10239B00040402020000000018244242424242425E
:1023AB004224180000000000080E0808080808085E
:1023BB0008083E00000000003C424242202010086A
:1023CB0004427E00000000003C42422018204040A6
:1023DB0042221C0000000000203028242422227EF0
:1023EB0020207800000000007E0202021A264040E6
:1023FB0042221C0000000000382402021A2642422E
:10240B0042241800000000007E2222101008080849
:10241B0008080800000000003C42424224182442F5
:10242B0042423C00000000001824424242645840E3
:10243B0040241C00000000000000001818000000E1
:10244B000018180000000000000000000800000049
:10245B0000000808040000004020100804020408D3
:10246B0010204000000000000000007F0000007FF3
:10247B0000000000000000000204081020402010A3
:10248B0008040200000000003C42424640201010AD
:10249B0000181800000000001C225A555555552DE8
:1024AB0042221C00000000000808181414243C22CF
:1024BB004242E700000000001F2222221E2242425D
:1024CB0042221F00000000007C4242010101010179
:1024DB0042221C00000000001F22424242424242A4
:1024EB0042221F00000000003F4212121E12120275
:1024FB0042423F00000000003F4212121E12120225
:10250B0002020700000000003C22220101017121A0
:10251B0022221C0000000000E7424242427E42425F
:10252B004242E700000000003E08080808080808BF
:10253B0008083E00000000007C1010101010101056
:10254B00101010110F0000007722120A0E0A12123F
:10255B0022227700000000000702020202020202A0
:10256B0002427F000000000077363636362A2A2AD0
:10257B002A2A6B0000000000E346464A4A52525298
:10258B0062624700000000001C2241414141414171
:10259B0041221C00000000003F424242423E020228
:1025AB0002020700000000001C2241414141414D45
:1025BB0053321C60000000003F4242423E12122286
:1025CB002242C700000000007C4242020418204057
:1025DB0042423E00000000007F4908080808080836
:1025EB0008081C0000000000E742424242424242FF
:1025FB0042423C0000000000E74242222424141413
:10260B0018080800000000006B4949494955553628
:10261B002222220000000000E7422424181818246C
:10262B002442E70000000000772222141408080857
:10263B0008081C00000000007E2120101008040474
:10264B0042423F00000078080808080808080808FC
:10265B00080808780000000202040408080810109B
:10266B002020204040001E101010101010101010D1
:10267B001010101E00003844000000000000000085
:10268B00000000000000000000000000000000003F
:10269B0000000000FF000608000000000000000022
:1026AB000000000000000000000000003C427844E5
:1026BB004242FC0000000000030202021A264242C2
:1026CB0042261A00000000000000000038440202FD
:1026DB000244380000000000604040407844424211
:1026EB004264D80000000000000000003C427E0263
:1026FB0002423C0000000000F08808087E08080831
:10270B0008083E0000000000000000007C22221C94
:10271B00023C42423C000000030202023A464242A3
:10272B004242E700000000000C0C00000E080808F5
:10273B0008083E0000000000303000003820202048
:10274B00202020221E0000000302020272120A1631
:10275B0012227700000000000E080808080808087D
:10276B0008083E0000000000000000007F929292DB
:10277B009292B70000000000000000003B4642426E
:10278B004242E70000000000000000003C424242D1
:10279B0042423C0000000000000000001B264242A9
:1027AB0042221E0207000000000000007844424253
:1027BB0042447840E000000000000000774C040425
:1027CB0004041F0000000000000000007C42023CDB
:1027DB0040423E0000000000000008083E080808C8
:1027EB000808300000000000000000006342424275
:1027FB004262DC000000000000000000E7422424DD
:10280B00140808000000000000000000EB494955C7
:10281B00552222000000000000000000762418184A
:10282B0018246E000000000000000000E742242482
:10283B001418080807000000000000007E22100892
:10284B0008447E000000C0202020202010202020E3
:10285B00202020C00010101010101010101010109D
:10286B0010101010100006080808080810080808B7
:10287B0008080806000C32C200000000000000002F
:0F288B000000000000000000000000000000003E
:00000001FF
